BL51 BANKED LINKER/LOCATER V6.22                                                        08/27/2014  12:19:42  PAGE 1


BL51 BANKED LINKER/LOCATER V6.22, INVOKED BY:
C:\KEIL\C51\BIN\BL51.EXE miaobiao.obj TO miaobiao


INPUT MODULES INCLUDED:
  miaobiao.obj (MIAOBIAO)


LINK MAP OF MODULE:  miaobiao (MIAOBIAO)


            TYPE    BASE      LENGTH    RELOCATION   SEGMENT NAME
            -----------------------------------------------------

            * * * * * * *   D A T A   M E M O R Y   * * * * * * *
            REG     0000H     0008H     ABSOLUTE     "REG BANK 0"

            * * * * * * *   C O D E   M E M O R Y   * * * * * * *
            CODE    0000H     008AH     ABSOLUTE     



SYMBOL TABLE OF MODULE:  miaobiao (MIAOBIAO)

  VALUE           TYPE          NAME
  ----------------------------------

  -------         MODULE        MIAOBIAO
  D:00F0H         SYMBOL        B
  C:0081H         SYMBOL        DELAY
  C:0046H         SYMBOL        DISPLAY
  B:00A8H.7       SYMBOL        EA
  B:00A8H.1       SYMBOL        ET0
  C:0083H         SYMBOL        LOOP1
  C:0076H         SYMBOL        LP
  C:0030H         SYMBOL        MAIN
  D:00A0H         SYMBOL        P2
  D:00B0H         SYMBOL        P3
  C:0064H         SYMBOL        T0_INTER
  C:0077H         SYMBOL        TAB
  D:008CH         SYMBOL        TH0
  D:008AH         SYMBOL        TL0
  D:0089H         SYMBOL        TMOD
  B:0088H.4       SYMBOL        TR0
  C:0000H         LINE#         2
  C:000BH         LINE#         4
  C:0030H         LINE#         6
  C:0033H         LINE#         7
  C:0036H         LINE#         8
  C:0039H         LINE#         9
  C:003CH         LINE#         10
  C:003EH         LINE#         11
  C:0040H         LINE#         12
  C:0042H         LINE#         13
  C:0044H         LINE#         14
  C:0046H         LINE#         15
  C:0047H         LINE#         16
  C:004AH         LINE#         17
BL51 BANKED LINKER/LOCATER V6.22                                                      08/27/2014  12:19:42  PAGE 2


  C:004BH         LINE#         18
  C:004CH         LINE#         19
  C:004EH         LINE#         20
  C:0050H         LINE#         21
  C:0053H         LINE#         22
  C:0055H         LINE#         23
  C:0057H         LINE#         24
  C:0058H         LINE#         25
  C:005AH         LINE#         26
  C:005CH         LINE#         27
  C:005FH         LINE#         28
  C:0061H         LINE#         29
  C:0064H         LINE#         30
  C:0067H         LINE#         31
  C:006AH         LINE#         32
  C:006BH         LINE#         33
  C:006EH         LINE#         34
  C:006FH         LINE#         35
  C:0071H         LINE#         36
  C:0074H         LINE#         37
  C:0076H         LINE#         38
  C:0081H         LINE#         40
  C:0083H         LINE#         41
  C:0085H         LINE#         42
  C:0087H         LINE#         43
  C:0089H         LINE#         44
  -------         ENDMOD        MIAOBIAO

Program Size: data=8.0 xdata=0 code=138
LINK/LOCATE RUN COMPLETE.  0 WARNING(S),  0 ERROR(S)
